:030000000208B043
:0C08B000787FE4F6D8FD7581500208F74F
:10099F000000415445300D0A000000000000000027
:1009AF000000000000000000000000000000000038
:1009BF0041542B43495053544152543D22544350B8
:1009CF00222C223139322E3136382E322E31303818
:1009DF00222C383038300D0A0041542B43495053E4
:0809EF00454E443D350D0A00A0
:100A3C00C103C102C1051E3300000000000000000C
:100A4C00000000000000000000000000000000009A
:100A5C00000000000000012300013200C100C101B0
:030A6C0001220064
:070B5D0053A27F43A2802296
:040B640053A27F22F7
:0E0B360000007F7F7EE97D94DDFEDEFCDFFAAD
:010B4400228E
:0E0B450000007F167E037DE3DDFEDEFCDFFA9E
:010B5300227F
:080B54007F0B7EF6DEFEDFFCE4
:010B5C002276
:100AEB0053877F759850438E40538EFE53890F4327
:0D0AFB008920758BFD758DFDC2ABD28E225A
:100A700020020330052A120B643005037550497BB0
:100A8000007A0079337D1E120AC77E007F1E7D002A
:100A90007B007A007933120A10C202C205120B5D84
:010AA0002233
:10093C00E4FFC206C207120B36120B36120B36122C
:10094C000AEBF59175923FD2ACD2AFD29C120B5DF3
:10095C00120B54120B54FFEF04FE74242FF8A6064E
:10096C000FBF0DF320060ED2067BFF7A0979A11278
:10097C000AA1120B36120A70300613200710D20788
:10098C007BFF7A0979BF120AA1120B36D203120A25
:03099C007080D197
:03002300020800D0
:09080000C0E0C0D075D000C000BA
:100809002098030208A2C298E521B40D1DE599B408
:100819000A18E5236401601220030F74342523F8B4
:100829007600D20275230075210074322523F8E67B
:10083900643A702A74312523F8E6643570207430DF
:100849002523F8E6B42C17742F2523F8E6B4440EB3
:10085900D3E523648094844005D2017522043001D4
:100869001ED3E522648094804004152280117434DB
:100879002523F8769FD202752300752200C20174E0
:10088900332523F8A6998599210523D3E523648087
:10089900949D4005752300D205309904C299C2047C
:0708A900D000D0D0D0E032F6
:060B230014F91209F7FFAE
:0D0B290030040122EFD204F5992004FD22D2
:100AA1008B0B8A0C890DAB0BAA0CA90D1209F760EF
:100AB10014120B54AB0B050DE50DAA0C7002050CBD
:060AC100120B2380E1226C
:100B08008B088A09890A7BFF7A0979E8120AA112F7
:0B0B18000B36AB08AA09A90A020AA1CB
:100AC7008B0B8A0C890DD3ED648094804015120B33
:100AD70054AB0B050DE50DAA0C7002050C120B2388
:040AE7001D80E32269
:1008BC0002093CE493A3F8E493A34003F68001F20D
:1008CC0008DFF48029E493A3F85407240CC8C3333D
:1008DC00C4540F4420C8834004F456800146F6DF0C
:1008EC00E4800B0102040810204080900A3CE47E56
:1008FC00019360BCA3FF543F30E509541FFEE49301
:10090C00A360010ECF54C025E060A840B8E493A3C7
:10091C00FAE493A3F8E493A3C8C582C8CAC583CAF2
:10092C00F0A3C8C582C8CAC583CADFE9DEE780BEAA
:010A6F000086
:1009F700BB010689828A83E0225002E722BBFE02FE
:090A0700E32289828A83E4932230
:100A1000EF4E6012EF60010EEDBB010B89828A83FD
:100A2000F0A3DFFCDEFA2289F05007F709DFFCA90A
:0C0A3000F022BBFEFCF309DFFCA9F02261
:00000001FF
